:100000000C942A001895000018950000189500001F
:10001000189500001895000018950000189500002C
:10002000189500001895000018950000189500001C
:10003000189500001895000018950000189500000C
:1000400018950000189500001895000018950000FC
:10005000189500008FE58DBFC0E2ECEA4E2E84E0DB
:100060008EBFD4E0F3E05F2EEEEFF3E0A0E6B0E069
:1000700088278D933197E9F76624899A9198889813
:100080008D9A8C988E9A9598AEE6B0E0E8E7FFE0FE
:100090000E94E806A2E7B0E0ECE7FFE00E94E80675
:1000A000E2E7F0E00E94C105EEE6F0E00E94BC0548
:1000B0000E942C06FF27EDE0A6E7B0E00E94B607FD
:1000C000E0E8FFE00E9493040E949B04EEEAFFE058
:1000D0000E949304A4E9B3E0E6E7F0E00E94BC05C7
:1000E0000E94CF040E949F040E949B04ECE6F0E073
:1000F000FA93EA935A924A9280E0A42DB52D8C93FC
:1001000081E00E94D9030E94E100249681E00E94D0
:10011000D503E2ECFFE00E949304A4E9B3E0ECE62F
:10012000F0E00E9458070E949F04EAE7F0E0FA938B
:10013000EA93ECE6F0E0FA93EA935A924A928DEF52
:1001400093E0A42DB52D8D939C9382E00E94D9035A
:100150005A924A928AE290E0A42DB52D8D939C93F9
:1001600082E00E94D903E6E7F0E0FA93EA930E9466
:1001700041012A9684E00E94D503EAECFFE00E9448
:100180009304A4E9B3E0AF93BF93EAE7F0E00E94E1
:10019000BC050E94CF0411E001E0BF91AF910E9425
:1001A000FD06E4E9F3E0A4E9B3E00E94B1070E9490
:1001B0009F040E949B0484EF91E00E94C0040C9471
:1001C000760000E010E020E030E0AFE7B0E00D9313
:1001D0001D932D933C9381E080937E0000917E00DF
:1001E000093018F011F00C942601ECE6F0E0FA93D7
:1001F000EA935A924A92AC81BD818C91A42DB52D7F
:100200008C9381E00E94D9030E948E01249681E0A4
:100210000E94D503AFE7B0E00D911D912D913C9167
:10022000ACE6B0E04D915C91662777270E944507C8
:10023000AFE7B0E00D931D932D933D93AEE7B0E093
:100240008C918F5F8C9310F40C94EE00AFE7B0E0CC
:100250000D911D912D913C9149E050E060E070E0DE
:100260000E941D04AFE7B0E04D935D936D937D93C5
:10027000AFE7B0E08D919C91AA81BB818D939C9357
:100280000895EC81FD81D190E080FF2400270E9439
:10029000E0050E9411062F933F934F935F93EE81E9
:1002A000FF81D190E080FF2400270E94E0055F914C
:1002B0004F913F912F910E948306FF27EDE0A3E825
:1002C000B0E00E94B607E881F9810E94C105E3E829
:1002D000F0E00E94BC050E942C06FF27EDE0A7E895
:1002E000B0E00E94B607E7E8F0E00E94C105EA81AD
:1002F000FB81D190E080FF2400270E94E0050E944E
:100300009206FF27EDE0ABE8B0E00E94B607EBE80D
:10031000F0E0A885B9850E94B6070895E2E9F0E00B
:10032000FA93EA930E9454022296A881B9810C9113
:10033000003011F00C94A501E2E9F0E0FA93EA93A1
:100340000E94540222960C94D701013011F00C94B3
:10035000B201E2E9F0E0FA93EA930E948B0222965E
:100360000C94D701023011F00C94BF01E2E9F0E0E7
:10037000FA93EA930E94C20222960C94D7010330AA
:1003800011F00C94CC01E2E9F0E0FA93EA930E94B8
:10039000F90222960C94D701043011F00C94D70185
:1003A000E2E9F0E0FA93EA930E943003229680E0BB
:1003B00090E0A0E9B0E08D939C9381E080938F0062
:1003C00000918F000C3018F011F00C943F02A881BE
:1003D000B9810C91003011F00C94F701E2E9F0E0E2
:1003E000FA93EA930E94540222960C942902013057
:1003F00011F00C940402E2E9F0E0FA93EA930E940F
:100400008B0222960C942902023011F00C941102F6
:10041000E2E9F0E0FA93EA930E94C20222960C9479
:100420002902033011F00C941E02E2E9F0E0FA9385
:10043000EA930E94F90222960C942902043011F0EA
:100440000C942902E2E9F0E0FA93EA930E94300367
:100450002296A0E9B0E00D911C91A2E9B0E04D9187
:100460005C91040F151FA0E9B0E00D931C93AFE859
:10047000B0E08C918F5F8C9310F40C94E001A0E9B4
:10048000B0E00D911C914CE050E00E940004A0E906
:10049000B0E04D935C93A0E9B0E08D919C91AA816E
:1004A000BB818D939C9308959598BB27A0E38C9175
:1004B00084FBDEF384E090E00E94C00480E090E0E2
:1004C000A2E9B0E08D939C93969A959A0027BB275A
:1004D000A0E38C9184FB0EF401E041E0041710F0DE
:1004E0000C948002A2E9B0E00D911C9141E050E033
:1004F000040F151FA2E9B0E00D931C930C94660243
:1005000095989698A2E9B0E08D919C91A881B981C7
:100510008D939C9308959598BB27A0E38C9184FBC1
:10052000DEF384E090E00E94C00480E090E0A2E965
:10053000B0E08D939C93969A959A0027BB27A0E3F1
:100540008C9184FB0EF401E041E0041710F00C9450
:10055000B702A2E9B0E00D911C9141E050E0040F18
:10056000151FA2E9B0E00D931C930C949D02959881
:100570009698A2E9B0E08D919C91A881B9818D9364
:100580009C9308959598BB27A0E38C9184FBDEF3A0
:1005900084E090E00E94C00480E090E0A2E9B0E036
:1005A0008D939C93969A959A0027BB27A0E38C91F4
:1005B00084FB0EF401E041E0041710F00C94EE020D
:1005C000A2E9B0E00D911C9141E050E0040F151F2D
:1005D000A2E9B0E00D931C930C94D40295989698E0
:1005E000A2E9B0E08D919C91A881B9818D939C93F3
:1005F00008959598BB27A0E38C9184FBDEF384E0FB
:1006000090E00E94C00480E090E0A2E9B0E08D9309
:100610009C93969A959A0027BB27A0E38C9184FB24
:100620000EF401E041E0041710F00C942503A2E958
:10063000B0E00D911C9141E050E0040F151FA2E9BC
:10064000B0E00D931C930C940B0395989698A2E937
:10065000B0E08D919C91A881B9818D939C93089570
:100660009598BB27A0E38C9184FBDEF384E090E0B7
:100670000E94C00480E090E0A2E9B0E08D939C93DA
:10068000969A959A0027BB27A0E38C9184FB0EF4E1
:1006900001E041E0041710F00C945C03A2E9B0E023
:1006A0000D911C9141E050E0040F151FA2E9B0E04C
:1006B0000D931C930C94420395989698A2E9B0E090
:1006C0008D919C91A881B9818D939C930895959863
:1006D000BB27A0E38C9184FBDEF384E090E00E94D2
:1006E000C00480E090E0A2E9B0E08D939C93969ADC
:1006F000959A0027BB27A0E38C9184FB0EF401E0C0
:1007000041E0041710F00C949303A2E9B0E00D91BE
:100710001C9141E050E0040F151FA2E9B0E00D93D9
:100720001C930C94790395989698A2E9B0E08D916A
:100730009C91A881B9818D939C9308959598BB272E
:10074000A0E38C9184FBDEF384E090E00E94C0047F
:1007500080E090E0A2E9B0E08D939C93969A959A00
:100760000027BB27A0E38C9184FB0EF401E041E05D
:10077000041710F00C94CA03A2E9B0E00D911C918B
:1007800041E050E0040F151FA2E9B0E00D931C9367
:100790000C94B00395989698A2E9B0E08D919C9145
:1007A000A881B9818D939C930895481A8827580A87
:1007B0000895480E8827581E089500FC10D008950B
:1007C00003D01ED001F8F9CF0024E89457FF02C0EF
:1007D00009D0689400F80BD010F80124089502D0D5
:1007E00009D00895509540954F5F5F4F0895E89464
:1007F00017FF0895009510950F5F1F4F6894089597
:10080000352F242FE894452B11F468940895512F27
:10081000402F0027112780E1440F551F001F111F93
:10082000021B130B416018F4020F131F4E7F8A95B1
:1008300099F7089500FC05D0089530D005D001F84F
:10084000F9CF37D03FD00895842F952FA62FB72FFB
:10085000E894452B462B472B11F468940895402FBC
:10086000512F622F732F0027112722273327F0E201
:10087000440F551F661F771F001F111F221F331FB4
:10088000081B190B2A0B3B0B416028F4080F191F9A
:100890002A1F3B1F4E7FFA9559F708950024E894CC
:1008A00077FF02C006D0689400F809D010F8012440
:1008B000089512D04F5F5F4F6F4F7F4F0895E894B8
:1008C00037FF089500951095209530950F5F1F4FC5
:1008D0002F4F3F4F689408954095509560957095BF
:1008E00008953197F1F70895689462F80895E894AF
:1008F00062F808958F939F9383E690E00197F1F754
:100900009F918F91089580952AE090E0089410F0CF
:10091000919802C0919A0000EDDFECDF96958795E3
:100920002A95A9F70895C895802D882319F0EBDF43
:100930003196F9CF08958DE0E6DF8AE0E4CFA4E9AF
:10094000B3E08D91882311F0DEDFFBCF08958F9304
:100950009F9383E690E00197F1F79F918F9108951F
:1009600029E0809BFECFF3DFF2DFF1DF88948099EE
:1009700008942A9519F087959795F6CF8095089554
:10098000EF93FF93EE27E82BE92B31F0E0EDF7E052
:100990003197F1F70197D1F7FF91EF9108958DE22B
:1009A00007FD8D938F2D881F802F881F8F57082F4D
:1009B0006894F7F8802F87FF15C080958395082FDE
:1009C00080E38D938EE28D93802F815228F080E317
:1009D0008D9399279C93089544270A95802F09F1B8
:1009E00096D01FC0805230F09EE49D9381E48D9399
:1009F0009D93EFCF4427DF92EF92FF920F938FE109
:100A0000801B11F0082F83D089D09EE29D930F9117
:100A1000FF90EF90DF9044270395003209F4D7CF81
:100A20002BD03F93EEEAFAE038E12F2D1E2D0D2D4D
:100A3000FF24EE24DD244427000F111F221FA8F4F9
:100A40002F923F920E94E006102C0E94E006202C7C
:100A50000E94E006302C0E94E0063197410DD21C26
:100A6000E31CF01C3F902F9001C0339631963A95CD
:100A700019F73F9107D0AFCFDD0CEE1CFF1C0A9594
:100A8000D9F70895002719E058D08F93802B11F0E3
:100A9000039501C08F911A95B9F7802F882309F427
:100AA00096CF8F91805D8D930A95D9F792CF00658F
:100AB000CD1D80B2E60E40597307A0ACB90350D6E5
:100AC000DC01286BEE0094357700CA9A3B0065CDB7
:100AD0001D00B2E60E0059730700ACB90300D6DC66
:100AE00001006BEE0000357700009A3B0000CD1D41
:100AF0000000E60E000073070000B9030000DC01EF
:100B00000000EE000000770000003B000000F694BB
:100B1000E794D79447950A95D1F7089500270DD00B
:100B20008F9303958F2D8E298D29842BC1F78F915B
:100B3000805D8D930A95D9F74CCF1F930F930027B3
:100B400010E2440FDD1CEE1CFF1C001F802F9AE0FA
:100B5000890B10F0082F43951A9599F7802F0F9164
:100B60001F910895D094E094F09491E0D90E9927C4
:100B7000E91EF91E10950895D190E190F190019130
:100B8000089521913191419151910895102F90E84C
:100B9000FF0C001F0927990FF7941078652F90E834
:100BA000440F551F5927990F4795607800380895CD
:100BB000FF0C90E89027110F9795F794092F08954F
:100BC000102FBD2CDE2CEF2CF02E11234AF4B09404
:100BD000D094E094F0949FEFB91AD90AE90AF90A7F
:100BE0000EE1FF2039F4FE2CED2CDB2CBB24085049
:100BF000C2F766C032F00A95BB0CDD1CEE1CFF1C70
:100C0000F9CF01D0D5CFB7FE089590E8B91611F409
:100C1000D0FE08959FEFD91AE90AF90A09F403955D
:100C20000895502F2D2D3E2D4F2D612F08952DEC21
:100C30003CEC4CEC5DE366270FC09EDFF2DFDD2469
:100C4000EE2490E8F92E0FE307C09BDF05C02227B2
:100C5000332740E251E46627552351F1002381F107
:100C600095DF71F11627005850580894050B18F4B9
:100C700007FD03C025C007FD23C04695379527957E
:100C8000F694E794D79422D0FF202AF0DD0CEE1CD6
:100C9000FF1C015073F09D2D969548F0DD203AF42D
:100CA000EE202AF491E0D90E9927E91EF91E80CF93
:100CB00007C09FE7092FF92A9FEFD92EE92E089543
:100CC000DD24EE24FF240027112708959F92992404
:100CD000AA24BB2488E1D216E306F40628F0D21A2F
:100CE000E30AF40A089401C08894991CAA1CBB1C4E
:100CF000DD0CEE1CFF1C8A9571F7D92CEA2CFB2C1D
:100D00009F9008953EDF42DF503829F090E8692730
:100D10000CC00AF045D04CCF5FE32227332744278D
:100D200001C02FDF33DF5038B1F3003899F3902F33
:100D3000951B8BF312F434D0FACF983118F0222798
:100D400033274427983028F0232F342F44279850F6
:100D5000F9CF992329F04695379527959A95D9F794
:100D6000912F962742F014D0B0F6F794E794D794D9
:100D70000F5F8BF69ECF10D051F008F4F3DEFF200A
:100D800052F2DD0CEE1CFF1C0150CBF792CF98CF36
:100D9000D20EE31EF41E0895D21AE30AF40A08954F
:100DA000DF92EF92FF920F931F93D22EE32EF42E39
:100DB000052F162F6F915F914F913F912F910895BD
:100DC000C89531960020089591E005C092E003C0D7
:100DD00094E001C098E0F4DF0D929A95E1F7089550
:100DE00099278D9193958823E1F7939511968C938C
:100DF00011978E919A95D1F70895EA2FFB2F002431
:100E00004C918D9103948E32E1F711248D911394BE
:100E10008823E1F71A94101640F41197202F211916
:100E2000239580E38D932A95E9F7113039F59927B9
:100E3000AE2FBF2FA00DB91FA00FB91F8C919C938F
:100E4000853308F421C031E08E918E32E9F38D3282
:100E500041F0830F8A3319F480E331E001C0332776
:100E60008C93AE1789F7332341F0AE2FBF2FB8DF35
:100E700081E34D3209F43196808308958827E00D8F
:100E8000F81FE00FF81F80830895040F151F261F19
:100E9000371F0895000F111F221F331F089500955B
:100EA0001095209530950F5F1F4F2F4F3F4F08959E
:100EB000019110810EC001911191219130810BC0DF
:100EC0000191108117FF05C03FEF2FEF04C0008193
:100ED00011272227332737FF03C0E1DF8DE28D93EF
:100EE000CF93DF93CF92DF92EF92AA24BB24CC243E
:100EF000DD24EE2440E2CAE0DD2755E093E388815B
:100F0000890F87FD9F7083FD907F891B89935A9578
:100F1000A9F7C0DFAA1CBB1CCC1CDD1CEE1C4A952B
:100F200051F7E894EFE0FF2782910ED0EB30E0F725
:100F30001EF068948A2D0CD088278D93EF90DF9057
:100F4000CF90DF91CF910895982F829501D0892F6E
:100F50008F70805D26F0803309F4089568948D9336
:100F6000089581918D938823E1F7089594E081910C
:100F70008D939A95E1F708950000C84200006842F9
:100F80006D3136382D746573742D636170616369DA
:100F9000746F722D72632D74696D696E672D64694B
:100FA000726563742E762E30322E62617300636E2A
:100FB00074207065722070657263656E74203D20C8
:100FC000000020326176673D000020617667253D94
:020FD00000001F
:00000001FF
